:100000000C943F040C94AB040C945D080C94AB046A
:100010000C94D4090C94AB040C94AB040C94AB0476
:100020000C94AB040C94AB040C94E71D0C94AB043F
:100030000C944A2C0C94AB040C94AB040C94AB04BD
:100040000C94AB040C94AB040C94AB040C94AB0474
:100050000C94AB040C949F2C0C94AB040C94AB0448
:100060000C94AB040C94AB040C94AB040C94AB0454
:100070000C94AB040C94AB040C94AB040C94AB0444
:100080000C94AB040C94AB040C94AB040C94AB0434
:100090000C94AB040C94AB040C94AB040C94AB0424
:1000A0000C94AB040C94AB040C94AB04110D1F0D19
:1000B0002B0D2B0D030D2B0D2B0D2B0D2B0D2B0DA8
:1000C0002B0D2B0D2B0D2B0D2B0D2B0D2B0D2B0D70
:1000D000050D2B0D070D2B0D2B0D2B0D2B0D230DB2
:1000E0002B0D3A0D210D2B0D2B0D2B0D2B0D2B0D4B
:1000F0002B0D2B0D2B0D2B0D2B0D2B0D2B0D2B0D40
:10010000FB0C170D090D1B0D2B0D0B0D2B0D0F0DE2
:100110002B0D190D0D0D1D0D130D150D2B0D2B0D8B
:100120002B0D2B0D2B0D2B0D2B0DFD0CFF0C010D95
:10013000250D270D2B0D2B0D2B0D290DD50DD70DB5
:10014000E30DE30DE30DE30DE30DE30DD90DDB0D41
:10015000DD0DE30DE30DD70DE60DE30DE30D9F0D72
:10016000D50DE30DE30DDB0DE30DE30DE30DE30D25
:10017000E30DE30DDD0DD50DC10DE30DC50DE30D53
:10018000E30DE30DA10DD90DE30DE30DCF0DE30D4F
:10019000E30DE30DA30DE10DE30DC30DE30DD70D4D
:1001A000E30DE30DD30DC70DE30DC90DDB0DE30D1D
:1001B000E30DE30DD10DCB0DE30DE30DE30DE30DE9
:1001C000E30DE30DE30DCD0DE30DA50DE30DE30D03
:1001D000D90DE30DE30DE10DE30DE30DE30DE30DAB
:1001E000E30DE30DE30DE30DE30DA70DE30DE30DCB
:1001F000E30DCF0DE30DE30DE30DE30DE30DE30D93
:10020000E30DE30DE30DE30DA90DE30DAB0DAD0D16
:10021000E30DE30DE30DAF0DB10DB30DE30DB50D22
:10022000B70DE30DE30DE30DDF0DB90DE30DBD0DCE
:10023000BB0DBF0DE30DE30DE30DE30DE10D280E46
:10024000760E510E9C0EC20ECA0ED10ED60EDA0ECE
:10025000710F730F750F770F790F810F810F810F5A
:100260007B0F7D0F7F0F59107A108E10AB10BD10D1
:10027000C810EC1005112B114D112312C813A6152F
:10028000351C5C1C541D5C1C541DA81CCB1C541D2F
:10029000221D311D372237226F226F22EA221E23B0
:1002A0001525152535231525C622C622CF2415254B
:1002B000E424022572253032582000522000643A8E
:1002C00025752000633A257520006973723A253040
:1002D0003458200077253032582000214353335FB3
:1002E0004630210A00214353335F5245414459218E
:1002F0000A00214353335F5245534554210A0021DC
:100300004353325F45305F4630210A002143533268
:100310005F46302120253032580A00214353325F96
:100320004530210A00214353325F494E4954210A86
:1003300000214353315F45305F25303258210A0098
:100340004D5B783A256420793A256420763A256415
:1003500020683A256420623A253032585D0A000A46
:100360005B434C525D20004C257520000A4D6F7593
:1003700073653A2025730A000A4445463A20000A6C
:100380004558503A20000A494E543A20000A4C4F32
:10039000473A20000A4C4D533A200053257520005F
:1003A0000A49443A253034582825732573292000FA
:1003B0000A556E6B6E6F776E2049443A2052657015
:1003C0006F727420746F20544D4B20004E472000F4
:1003D0004F4B20000A353537365F43533832683A81
:1003E00000522575200057257520005725752000DF
:1003F0005725752000582575200041257520004996
:10040000257520005B4348475D20000A2575205074
:1004100052543A25303258204953523A25303458F4
:1004200020005B5253545D20000A2575204552522E
:100430003A25303258204953523A2530345820005A
:10044000535B253032582025303258202530325821
:100450005D2000007B46010203763A687F6577489D
:100460002B353B6978796439141E3C6A7A1D160471
:100470001A1F3D6B061B070821203E6C2C1909171B
:1004800015223F6D11050B0A1C23406E7E100D18BE
:100490002425416F360E0C122726427037380F3351
:1004A000132D43717534322F2E44727C7D283031E8
:1004B00074457351504A524D492A5466594F5C5FF6
:1004C0004C4B4E62635A5D5E60295367585B5657CA
:1004D0006147554842403E3C3A3B456843413F3DB9
:1004E0002B357E697A790078141E7C6A7B1D160490
:1004F0001A1F7F6B061B070821204D6C2C1909174A
:1005000015224A6D11050B0A1C234C6E49100D185B
:100510002425516F360E0C1227264F7037380F33B3
:10052000132D52717534502F2E4E72397D2830653F
:10053000314B735464586776012A773259745C5F83
:1005400066020362635A5D5E60295344575B5655E9
:1005500061474680291E1F20212223242526272D7E
:100560002E2A2B141A0815171C180C12132F3028BA
:1005700078041607090A0B0D0E0F33343579311D37
:100580001B06190511103637387D557A2C393A3B40
:100590003C3D3E3F4041424353475F6061565C5D96
:1005A0005E57595A5B62634648644445677B7F6582
:1005B0000301025250514F68696A6B6C6D6E6F7027
:1005C00071725800494C754A4D734B4E767C777E5C
:1005D0007466540A4C6F6F702073746172742E0AC3
:1005E000000A55534220636F6E66696775726564D1
:1005F0002E0A000A544D4B3A3464366537662F4C48
:100600005546413A6436613764660A00340349004E
:1006100042004D0020005000430020006B006500A8
:10062000790062006F0061007200640020006300C6
:100630006F006E0076006500720074006500720045
:100640000000080354004D004B000000040309049F
:1006500009025B00030100A032090400000103014C
:100660000100092111010001223900070581032041
:100670000001090401000103010200092111010028
:1006800001227F000705820308000109040200021D
:100690000300000009211101000122220007058347
:1006A00003200001070503032000011201100100CF
:1006B000000008EDFEEE1B0102010200010631FF01
:1006C0000974A1010975150026FF009520750881A0
:1006D000020976150026FF00952075089102C005D5
:1006E000010902A1010901A10085010509190129DA
:1006F00008150025019508750181020501093009D9
:10070000311581257F9502750881060938158125E7
:100710007F950175088106050C0A38021581257F31
:10072000950175088106C0C005010980A1018502F7
:100730001601002637001A81002AB70075109501AE
:100740008100C0050C0901A1018503160100269C4A
:10075000021A01002A9C02751095018100C0050152
:100760000906A101050719E029E7150025019508EB
:100770007501810205081901290595057501910288
:100780009501750391010507190029F71500250149
:1007900095F875018102C0636F6E73756D65723A6D
:1007A00020253034580A0073797374656D3A20251A
:1007B0003034580A000A002530325820006B657921
:1007C000626F6172643A20004C45443A2025303211
:1007D000580A0025583A253031366225730A000A36
:1007E00020203031323334353637383941424344B2
:1007F00045460A0064656C5F6B65795F6269743AAF
:100800002063616E27742064656C3A20253032586D
:100810000A006164645F6B65795F6269743A2063A2
:10082000616E2774206164643A20253032580A00D2
:10083000290A002575002F002575005D2800256414
:1008400000200025640020002564002000256400AD
:100850007C0025303258006D6F7573656B657920AB
:100860005B62746E7C782079207620685D287265E2
:10087000702F61636C293A205B004B0B0916112421
:100880001FBECFEFDAE0DEBFCDBF04B603FE41C02E
:100890008091210490912204A0912304B09124041A
:1008A0008730904BA740B04BA1F5109221041092D5
:1008B0002204109223041092240414BE0FB6F8945C
:1008C000A89580916000886180936000109260001C
:1008D0000FBE1092010810920008E3E0F0E089E0FA
:1008E00080935700E491E695E370E150E33040F4E3
:1008F000F0E0EE0FFF1FE858FE4F8081918102C0AB
:1009000080E090E1E0E0F0E8E81BF90BF695E79570
:10091000099511E0A0E0B1E0ECEEF1E602C005902F
:100920000D92AE37B107D9F724E0AEE7B1E001C0D0
:100930001D92A132B207E1F714E0CFE3D4E004C086
:100940002197FE010E94DA30CD33D107C9F70E940A
:1009500048190C94F4300C940000FF93EF93E0914D
:100960007E01F0917F01309709F00995EF91FF9199
:100970000895FC018591803011F0EFDFFBCF0895E1
:10098000FF27E0E230E247FF0CC0419597FF09C026
:10099000EDE26095709580959095611D711D811DAA
:1009A000911D27FF02C0219530E350E2AA27660F70
:1009B000771F881F991FAA1FA41710F0A41B639507
:1009C0005A95A9F7AA3008F0A95FA05DAF93F395F7
:1009D000611571058105910541F7ED3211F4EF9331
:1009E000F395F21718F43F93F395FBCF8F91B5DF92
:1009F000FA95E1F70895E991F9918591803021F018
:100A0000853219F0AADFF9CF089520E0E8945591D6
:100A10005532C1F3503311F4689455915A3348F468
:100A2000505390F3220F022E220F220F200D250F7C
:100A3000F4CF0EF4219589919991533619F35337D8
:100A400029F1533559F1BC0188279927E8945C3680
:100A500021F48991999168945591543639F446EF6F
:100A60007EF077FF0DC08FEF9FEF0AC055374AE049
:100A700039F0583540E121F0523642E009F008954E
:100A8000FF93EF937DDFEF91FF91B7CFFF93EF934C
:100A9000FC0181918030B9F360DFFBCFFF93EF93CE
:100AA00068DFF1CFDF93CF93CDB7DEB72596A3DF15
:100AB000CF91DF910895FC012AB1938D90959223F7
:100AC0009AB99BB1838D892B8BB90895FC019AB19A
:100AD000838D809589238AB99BB1838D892B8BB9AE
:100AE00085E08A95F1F7000099B1838D982381E024
:100AF00009F480E00895FC012BB1948D9095922328
:100B00009BB99AB1848D892B8AB90895FC012AB1C9
:100B1000948D909592239AB99BB1848D892B8BB932
:100B20000895FC019AB1848D809589238AB99BB17F
:100B3000848D892B8BB985E08A95F1F7000099B1F6
:100B4000848D982381E009F480E008950F931F932A
:100B5000CF93DF938C01EB01C8010E9466058823C7
:100B600041F0209731F085E08A95F1F70000219758
:100B7000F3CFCE01DF91CF911F910F9108950F9385
:100B80001F93CF93DF938C01EB01C8010E94660590
:100B9000811108C0209731F085E08A95F1F70000B7
:100BA0002197F3CFCE01DF91CF911F910F9108953F
:100BB0000F931F93CF93DF938C01EB01C8010E9429
:100BC0009105811108C0209731F085E08A95F1F7F1
:100BD00000002197F3CFCE01DF91CF911F910F91AC
:100BE0000895CF93DF93EC010E945B05CE01DF9166
:100BF000CF910C9486053BB1FC01238D20952323D6
:100C00002BB93AB1238D232B2AB90C948605FC010C
:100C10008CB3938D982B9CBB9DB3838D892B8DBBFF
:100C20000895CF93DF93EC010E940706CE01DF9178
:100C3000CF910C94F105FC012DB3938D90959223E7
:100C40009DBBCF010C94FB05FC0111821082128226
:100C5000138280E090E8958384831782108608953C
:100C6000CF93DF93EC012E9826982F9827980E9417
:100C7000FB05898D843080F440916900880F22E063
:100C800030E0B90102C0660F771F8A95E2F7CB0109
:100C9000842B8093690010C040916A008370880F94
:100CA00022E030E0B90102C0660F771F8A95E2F7B3
:100CB000CB01842B80936A009DB38B8D8095892313
:100CC0008DBBCE01DF91CF910C942406CF93DF939F
:100CD000EC018F8190E001968F709927288530E094
:100CE0008217930749F4CE010E942406CE010E9488
:100CF0000706CE010E94F1052FB7F89498858F81E1
:100D0000891751F0FE01E90FF11D81859F5F9F70EA
:100D10009887C82FD0E002C0CFEFDFEF2FBFCF3FC3
:100D20008FEFD80781F08091060480FF0CC0DF931D
:100D3000CF9384EB92E09F938F930E9452050F9084
:100D40000F900F900F90CE01DF91CF9108950F93E8
:100D50001F93CF938C01CAE1C15071F0C8010E946A
:100D600066068F3F2FEF920749F48FE99FE00197C6
:100D7000F1F700C00000F0CF8FEF9FEFCF911F91F0
:100D80000F9108952F923F924F925F926F927F92B0
:100D90008F929F92AF92BF92CF92DF92EF92FF928B
:100DA0000F931F93CF93DF93EC01062F1B8280914B
:100DB000060480FF0CC01F926F9384ED92E09F9316
:100DC0008F930E9452050F900F900F900F908C817F
:100DD0009D818115904891F08091060480FF0EC09E
:100DE0008C819D819F938F938AEC92E09F938F9348
:100DF0000E9452050F900F900F900F908C819D8153
:100E000081159048D9F7CE010E946605811115C061
:100E10008091060480FF11C068EE73E0CE010E944D
:100E2000BF059F938F9384EC92E09F938F930E94D2
:100E300052050F900F900F900F90CE010E949105D8
:100E4000811115C08091060480FF11C068EE73E027
:100E5000CE010E94D8059F938F938EEB92E09F93D3
:100E60008F930E9452050F900F900F900F909DB39B
:100E70008B8D809589238DBB9BE0D92ECC24C39488
:100E800010E09924939428E0222E37E0332E46E098
:100E9000842E55E0752E64E0662E73E0572EE2E056
:100EA0004E2EFBEBAF2EF2E0BF2ECE010E94FB05D3
:100EB0008FE193E00197F1F700C00000CE010E949E
:100EC0007B058FE193E00197F1F700C00000CE01B0
:100ED0000E945B0560E177E2CE010E94A605892BA6
:100EE00011F49B826AC0E12CF12C90E59A95F1F700
:100EF000C8010E2C02C0959587950A94E2F780FFF1
:100F000005C0C924CE010E94860503C0CE010E94FF
:100F10007B0562E370E0CE010E94BF05892B11F4CE
:100F20004B824BC062E370E0CE010E94A605892B84
:100F300011F45B8242C02FEFE21AF20A88E0E81651
:100F4000F10499F690E59A95F1F7CE01CC2019F0CD
:100F50000E94860502C00E947B0562E370E0CE011C
:100F60000E94BF05892B11F46B8227C062E370E0F9
:100F7000CE010E94A605892B11F47B821EC020E5BC
:100F80002A95F1F7CE010E9486058CE2E82EFF2417
:100F9000F394CE010E949105882329F0E114F10415
:100FA000D9F58B820AC0EF28E1F36CE271E0CE0143
:100FB0000E94D805892B49F43B828B81813009F04E
:100FC0003FC0DA94D11030C03BC06CE271E0CE017A
:100FD0000E94BF05892B11F42B82EFCFCE010E9416
:100FE0002406CE010E94F105CE010E940706CE0123
:100FF000DF91CF911F910F91FF90EF90DF90CF90F5
:10100000BF90AF909F908F907F906F905F904F9028
:101010003F902F900C94A70685E08A95F1F7000089
:1010200091E0E91AF108B5CF1B828091060480FF98
:101030003CCFBF92AF920E9452050F900F9035CFD8
:101040008B8180618B83CE010E94FB058FE39FE142
:101050000197F1F700C00000CE010E94F105CE011A
:101060000E9407068FEF9FEFDF91CF911F910F91A5
:10107000FF90EF90DF90CF90BF90AF909F908F90B8
:101080007F906F905F904F903F902F9008951F93A7
:10109000CF93DF93EC01162F6DEE0E94C2068A3FBC
:1010A000910539F4612FCE01DF91CF911F910C94FE
:1010B000C206DF91CF911F9108951F920F920FB634
:1010C0000F9211242F933F934F935F938F939F938E
:1010D000EF93FF9349B15091B7019091070420918C
:1010E000A1013091A2012115304819F49093A30178
:1010F0000FC08091A301981B933050F08091A10103
:101100009091A20190939E0180939D0180E21EC167
:101110002091A1013091A201369527953093A2012B
:101120002093A10181E090E001C0880F5A95EAF771
:10113000842349F08091A1019091A201906890933D
:10114000A2018093A1018091A1019091A201992710
:101150008038910509F41BC1A8F48032910509F487
:1011600016C138F4009709F412C1409709F495C0EC
:10117000B5C08034910509F40AC18035910509F4A0
:101180008CC0ACC0803C910531F148F480399105A8
:1011900009F483C0803A910509F44DC09FC0803D99
:1011A000910509F47AC0803E910509F097C08091BD
:1011B000A1019091A20190939E0180939D01809145
:1011C000A1019091A201892F99279093A201809368
:1011D000A10183E256C080919F01811123C084E662
:1011E00029B19091B801922311F48111B8C029B1AD
:1011F0009091B8019223E1F08111B7C08091A101D3
:101200009091A20190939E0180939D018091A101F4
:101210009091A201892F99279093A2018093A10117
:1012200082E22FC080919F01823209F0B0C0E6CFE8
:101230008111ADC0E3CF80919F01811125C084E66B
:1012400029B19091B801922311F4811194C029B170
:101250009091B8019223F1F0811193C08091A10186
:101260009091A20190939E0180939D018091A10194
:101270009091A201892F99279093A2018093A101B7
:1012800081E280939F0136C080919F01813209F0F5
:101290007EC0E4CF81117BC0E1CF8091A10190910C
:1012A000A20190939E0180939D018091A101909154
:1012B000A20197FF02C080E101C081E180939F01FC
:1012C0008091A1019091A20126E0969587952A959B
:1012D000E1F79093A2018093A1010CC010929F01AD
:1012E0008091A1019091A20190939E0180939D0114
:1012F00080E82CC02091A1013091A2018091A4012D
:10130000E82FF0E0E356FE4F21878F5F8F708093C8
:10131000A40190E001968F7099273091A501432F89
:1013200050E08417950769F42DB38091B801482FD8
:10133000409524232DBB9BB194239BB99AB1892B53
:101340008AB98091A401831303C080E48093A00133
:1013500080E090E89093A2018093A10118C095E0ED
:101360009A95F1F7000081503BCF95E09A95F1F7FF
:10137000000081503CCF95E09A95F1F70000815034
:101380005FCF95E09A95F1F70000815060CFFF9113
:10139000EF919F918F915F914F913F912F910F907E
:1013A0000FBE0F901F9018951F920F920FB60F92BD
:1013B00011242F933F934F935F938F939F93EF93BA
:1013C000FF9349B150919A019091070420918401B3
:1013D000309185012115304819F4909386010FC092
:1013E00080918601981B933050F0809184019091F8
:1013F0008501909381018093800180E21EC120913C
:10140000840130918501369527953093850120938D
:10141000840181E090E001C0880F5A95EAF78423A7
:1014200049F08091840190918501906890938501A5
:10143000809384018091840190918501992780385F
:10144000910509F41BC1A8F48032910509F416C175
:1014500038F4009709F412C1409709F495C0B5C05B
:101460008034910509F40AC18035910509F48CC0D6
:10147000ACC0803C910531F148F48039910509F404
:1014800083C0803A910509F44DC09FC0803D91050D
:1014900009F47AC0803E910509F097C080918401DB
:1014A00090918501909381018093800180918401C6
:1014B00090918501892F99279093850180938401CC
:1014C00083E256C080918201811123C084E629B154
:1014D00090919B01922311F48111B8C029B1909190
:1014E0009B019223E1F08111B7C08091840190911A
:1014F0008501909381018093800180918401909176
:101500008501892F9927909385018093840182E238
:101510002FC080918201823209F0B0C0E6CF8111E4
:10152000ADC0E3CF80918201811125C084E629B14D
:1015300090919B01922311F4811194C029B1909153
:101540009B019223F1F0811193C0809184019091CD
:101550008501909381018093800180918401909115
:101560008501892F9927909385018093840181E2D9
:101570008093820136C080918201813209F07EC061
:10158000E4CF81117BC0E1CF8091840190918501EE
:1015900090938101809380018091840190918501D5
:1015A00097FF02C080E101C081E1809382018091B8
:1015B00084019091850126E0969587952A95E1F71B
:1015C00090938501809384010CC0109282018091D8
:1015D000840190918501909381018093800180E83E
:1015E0002CC0209184013091850180918701E82FE2
:1015F000F0E0E058FE4F21878F5F8F708093870166
:1016000090E001968F70992730918801432F50E028
:101610008417950769F42DB380919B01482F40955D
:1016200024232DBB9BB194239BB99AB1892B8AB9F2
:1016300080918701831303C080E48093830180E05D
:1016400090E8909385018093840118C095E09A9565
:10165000F1F7000081503BCF95E09A95F1F700003B
:1016600081503CCF95E09A95F1F7000081505FCF13
:1016700095E09A95F1F70000815060CFFF91EF91CE
:101680009F918F915F914F913F912F910F900FBE3E
:101690000F901F901895EDE9F1E0118210821282EF
:1016A000138220E030E835832483168291E0918F05
:1016B000128E82E0838F948FE0E8F1E01182108235
:1016C0001282138235832483168293E0918F828F56
:1016D00088E0838F84E0848F0895262F30E094E0A3
:1016E000359527959A95E1F72770E62FEF708230B0
:1016F00069F08330A1F08130E1F4F0E080E1289FCF
:10170000E00DF11D1124ED5AFA4F11C0F0E080E117
:10171000289FE00DF11D1124ED52FB4F08C0F0E0B1
:1017200080E1289FE00DF11D1124ED5AFB4F8491BB
:10173000089580E808950F931F93CF93DF938C0152
:10174000EB0169EEFC01808191810E94C206F801E3
:10175000808191810E94A7068883F8018081918110
:101760000E94A7068983F801808191810E94A706C3
:101770008A8399279F938F9389811F928F93888162
:101780001F928F9380E494E09F938F930E94520561
:101790008DB79EB708960FB6F8949EBF0FBE8DBF4B
:1017A000DF91CF911F910F910895E6EDF1E0119235
:1017B000119281E0E63EF807D1F708951F93CF9389
:1017C000DF93FC0184810E946D0B87FD20C0182FE0
:1017D0001F70C82FD0E094E0D595C7959A95E1F792
:1017E000612F8C2F0E945120811111C0CC0FDD1F61
:1017F000CA52DE4F81E090E002C0880F991F1A950F
:10180000E2F728813981822B932B99838883DF919A
:10181000CF911F9108951F93CF93DF93FC01848193
:101820000E946D0B87FD22C0182F1F70C82FD0E0BB
:1018300094E0D595C7959A95E1F7612F8C2F0E947A
:101840005120882399F0CC0FDD1FCA52DE4F81E072
:1018500090E002C0880F991F1A95E2F78095909545
:10186000288139818223932399838883DF91CF91C3
:101870001F9108958091C8019091C9010E9430067E
:101880008091BA019091BB010C94300680910604BE
:101890008160809306040C94D50BE82FF0E0EE0FE6
:1018A000FF1FEA52FE4F8081918108950C94D50B61
:1018B0007770E72FF0E098E0899FE00DF11D11248B
:1018C00084E0EE0FFF1F8A95E1F76F70E60FF11DC0
:1018D000EE0FFF1FE050F849859194910895FC01A7
:1018E0008481823070F0843061F062FB992790F936
:1018F00060FD926061FD9460692F808191810C94FC
:1019000047080895CF93C82F682F88EC91E00E9474
:101910006F0C6C2F8AEB91E0CF910C946F0CCF92EF
:10192000DF92EF92FF920F931F93CF93DF936C019F
:101930008B010E94782C7C01F601808191810E94AC
:101940006606EC01019631F4C7010E94902C8017C5
:10195000910790F3CE01DF91CF911F910F91FF90EE
:10196000EF90DF90CF9008950F931F93CF93DF9365
:10197000FC0180819181DC0112962C912131F9F0DA
:101980008F0162EF0E94C2068F3FBFEF9B07D1F02D
:101990008A3F9105D1F464EF71E0C8010E948F0C79
:1019A0008F3F2FEF9207A1F0D82FCC2764EF71E083
:1019B000C8010E948F0CDE01A82BCD010BC08DEF5A
:1019C0009FEF08C08FEF9FEF05C08EEF9FEF02C023
:1019D00080E090E0DF91CF911F910F910895CF9318
:1019E000862F90E0FC017C97E834F105A0F5EA5AD7
:1019F000FF4F0C94DA3085E53EC08AE53CC08BE5AC
:101A00003AC08CE538C08DE536C08EE534C08FE530
:101A100032C080E630C081E62EC082E62CC083E66C
:101A20002AC08FE628C081E726C082E724C084E769
:101A300022C085E720C087E71EC088E71CC08AE770
:101A40001AC08CE718C08FE716C080E714C089E77A
:101A500012C08BE710C0C62F1F926F9381E393E0F3
:101A60009F938F930E9452050F900F900F900F90AD
:101A70008C2F01C084E5CF910895CF93DF93EC01C3
:101A800099859230A9F128F4992341F09130C9F059
:101A900045C09330B1F19430D9F140C0603E21F09F
:101AA000613E21F482E02BC081E029C067FD04C0C3
:101AB000CE010E94DE0B33C06F77CE010E940B0C6B
:101AC0002EC0663359F118F46A3229F427C06A3AF5
:101AD00029F1663B19F167FD05C0CE010E94EF0CAC
:101AE000682F12C06F77CE010E94EF0C682F13C0D1
:101AF0006D3121F06D3991F484E001C083E0898774
:101B00000EC0653459F465E5CE010E94DE0B06C0B7
:101B1000653C21F465E5CE010E940B0C198680E03E
:101B2000DF91CF910895862F90E0FC013397E13843
:101B3000F10508F048C0E256FF4F0C94DA3087E117
:101B400008958FE108958CE5089580E6089582E672
:101B5000089587E2089583E508958FE2089589E363
:101B6000089587E308958FE3089587E408958FE447
:101B7000089586E508958EE508958FE7089580E03D
:101B8000089585E608958EE608958FE6089580E32A
:101B9000089588E3089580E4089588E4089580E531
:101BA000089587E508958FE5089588E1089588E010
:101BB000089580E2089580E1089589E108958DE611
:101BC000089588E20895862F8F7708958FE008950D
:101BD0006B35C9F068F46131F1F020F46E30C9F46E
:101BE00084E50895633169F0643599F48BE50895CF
:101BF0006D3559F050F0623651F06C3751F487E78B
:101C0000089581E108958DE508958AE608958EE0AE
:101C10000895862F08958FE00895613131F0613481
:101C200011F48CE70895862F089583E108951F939A
:101C3000CF93DF93EC01162FEA858E2F90E0893049
:101C4000910508F0BDC0FC01E15EFE4F0C94DA3056
:101C50008A819B8180599B4A029720F4CE010E9481
:101C6000E80D182F103E69F030F4133871F0143875
:101C700071F46FE792C0113E31F0103F41F481E002
:101C800093C082E091C084E08FC062E086C01A8673
:101C900017FD02C0612F21C00E94D50B85E293E0A1
:101CA00069C08A819B8180599B4A029720F4CE01AA
:101CB0000E940D0E182F193509F482C0103F19F03B
:101CC000123119F47DC083E06FC01A8617FD09C078
:101CD000612FCE010E94930D682FCE010E94DE0B72
:101CE00070C00E94D50B8BE193E044C08A819B8138
:101CF00080599B4A029720F4CE010E94E80D182FCC
:101D0000133821F0143821F46FE757C062E055C052
:101D10001A8617FD02C0612F25C00E94D50B1F92A5
:101D20001F938CE093E09F938F930E9452050F9036
:101D30000F900F900F9024C08A819B8180599B4AFD
:101D4000029720F4CE010E940D0E182F1A86123130
:101D5000C1F11935B1F117FD09C0612FCE010E9403
:101D6000930D682FCE010E940B0C2BC00E94D50B47
:101D70008FEF92E09F938F930E9452050F900F90E8
:101D80008FEF20C0643121F0603FD1F486E00CC0B9
:101D900085E00AC06737A1F460E0CE010E94DE0B47
:101DA0000FC0643169F487E08A870BC0603F41F45B
:101DB00088E0FACF673721F460E0CE010E940B0C77
:101DC0001A8680E0DF91CF911F9108956C3551F014
:101DD00018F4633169F00AC0663731F06E3731F4B8
:101DE00086E7089581E508958EE70895862F089582
:101DF0008DE50895CF93DF93EC016F3B41F028F41C
:101E000086E5860F823070F402C06C3F59F41B8661
:101E100082EF92E09F938F930E9452050F900F9054
:101E20008FEFB1C08B85813009F445C038F0823026
:101E300009F476C0833009F491C0A4C08A819B81E3
:101E400082399B4A21F4CE010E94E60E682F663843
:101E500009F168F46338D1F020F4603819F582E0B4
:101E600077C06438A9F06538E9F468E61DC06C38BD
:101E7000A9F030F4673881F06B38A1F461E014C048
:101E80006D3871F0603F71F481E062C062E00CC0B7
:101E90006FE70AC068E708C060E006C069E004C0F8
:101EA0006AE002C067FD04C0CE010E94DE0B6AC07A
:101EB00085EE92E02EC01B868A819B8182399B4AE7
:101EC00021F4CE010E94E60E682F862F90E0FC01DF
:101ED000E358F109EB30F105A0F4E85DFE4F0C94F6
:101EE000DA3062E010C06FE70EC068E60CC068E749
:101EF0000AC060E008C061E006C069E004C06AE0B2
:101F000002C067FD04C0CE010E940B0C3BC08BEDEC
:101F100092E09F938F930E9452050F900F9032C0D2
:101F2000653279F030F4663171F06E3199F460E029
:101F30000BC0663221F0603F69F483E009C06DE5B3
:101F400003C063E501C061E5CE010E94DE0B04C061
:101F50008B8718C00E94D50B1B8614C06E3169F0A8
:101F600020F46631B9F761E509C0653221F06632C7
:101F700089F76DE503C063E501C060E0CE010E9412
:101F80000B0CEACF80E0DF91CF9108958F929F9262
:101F9000AF92BF92CF92DF92EF92FF920F931F9377
:101FA000CF93DF9300D000D01F92CDB7DEB78C0166
:101FB000DC01ED91FC9183818823B1F1E080F18017
:101FC000D3800E94782CFF92EF921F92DF929F9312
:101FD0008F9389E294E09F938F930E945205D801DA
:101FE000ED91FC911197838180750FB6F894DEBF57
:101FF0000FBECDBF81F418968C918B3061F482E2D4
:1020000094E09F938F930E9452058CE0D80118961C
:102010008C930F900F90D801ED91FC911197138242
:10202000ED91FC9111821082D801ED91FC911197F4
:102030008281882381F1928115968C91981759F1AC
:10204000E080F180D2800E94782CFF92EF921F9264
:10205000DF929F938F938BE094E09F938F930E94E6
:102060005205F80185810FB6F894DEBF0FBECDBFD3
:102070000190F081E02D85FF03C0928194FD6FC532
:1020800084FD6AC5D801ED91FC9111978281159666
:102090008C9311821082D8011896EC918E2F90E0CB
:1020A0008D30910508F09AC5FC01ED5CFE4F0C9453
:1020B000DA300E94782C9F938F938FEF93E09F9359
:1020C0008F930E945205F8011482138212821582A6
:1020D0000E94D50B0E94782CD80117969C938E9362
:1020E000169781E018968C9318978D919C910E9479
:1020F00011066DC0F801808191810E9466060196EB
:10210000C9F7D80116968D919C9117970E94902C33
:10211000893B9B4008F462C582E018C00E94782C7D
:102120009F938F938AEF93E09F938F930E94520522
:102130006FEFD8018D919C910E94C2060F900F9075
:102140000F900F908A3F910521F486E0F801808777
:1021500045C583E060C3F801808191810E941B0620
:102160002E98269A2F98279A0E94782CD801179695
:102170009C938E93169784E04FC3F80186819781D4
:102180000E94902C853F914008F428C585E043C308
:102190002E9826982F982798F801808191810E9487
:1021A0002406D8018D919C910E9411060E94782CE2
:1021B0009F938F9385EF93E09F938F930E94520597
:1021C0000E94782CF8019783868386E080870F90A1
:1021D0000F900F900F9002C5D8018D919C910E9495
:1021E0006606019609F4FAC40E94782C9F938F9397
:1021F00080EF93E09F938F930E9452050E94782C6A
:10220000F8019783868387E0E1CFD80116968D91F8
:102210009C9117970E94902C853F914018F089E07F
:10222000F8018087D8018D919C910E9466060196E5
:1022300009F4D4C40E94782C9F938F938BEE93E083
:102240009F938F930E9452050E94782CF8019783E8
:10225000868388E0BBCFD80116968D919C91179705
:102260000E94902C853F914018F089E0F80180870A
:10227000D8018D919C910E946606019609F4AEC426
:102280000E94782C9F938F9386EE93E09F938F9379
:102290000E94520589E0F80199CFC8010E94B40C50
:1022A000D80113969C938E9312970E94782C9F933B
:1022B0008F9381EE93E09F938F930E945205F801D4
:1022C000828193810F900F900F900F90009711F4DF
:1022D00082E010C08F3FBFEF9B0711F481E044C044
:1022E0009C012D5F3F4F2230310590F38F3F9105C8
:1022F00029F484E0D80114968C9363C09C0125587E
:102300003B4A2230310508F445C48239BBEA9B07B9
:1023100009F440C49C0120593B4A22303105F8F4AD
:1023200084ED93E09F938F930E94520560EFF80134
:10233000808191810E94C2060F900F908A3F910583
:1023400009F01FC462E8D8018D919C910E94C206D9
:102350008A3F910509F015C480ED93E014C4803BD9
:10236000BFEB9B0721F483E0F80184832AC0882710
:102370008115FBEA9F0709F4ABCF81152FEB92077C
:1023800091F381159F4779F380EB93E09F938F93AF
:102390000E94520560EFD8018D919C910E94C20667
:1023A0000F900F908A3F910509F0F4C362E0F801A5
:1023B000808191810E94C2068A3F910509F0EAC39B
:1023C00087CFF801228133812E3FFFEF3F0751F085
:1023D0002D3F4FEF340749F02115310549F040E218
:1023E00051E008C041E251E005C04BE151E002C0BC
:1023F00047E251E0D80114968C91813049F0823047
:1024000051F0833059F0843061F08CE391E00BC0DF
:1024100080E391E008C08DE291E005C083E391E0A4
:1024200002C081E491E05F934F939F938F933F931A
:102430002F9380EA93E09F938F930E9452058AE046
:10244000F80180877DC30E94782C9F938F938BE93E
:1024500093E09F938F930E9452050F900F900F90DF
:102460000F90D80114968C91833031F0843079F03C
:10247000823009F07CC106C068EFF801808191814B
:102480000E94C2060E94D51E0E94820C70C165EF98
:10249000D8018D919C910E94C2066AEEF80180815C
:1024A00091810E94C206BE016F5F7F4FC8010E94EA
:1024B0009B0B84E993E09F938F930E94520568EEF3
:1024C000D8018D919C910E94C20660E0F801808144
:1024D00091810E94C20666EED8018D919C910E9466
:1024E000C20666EEF801808191810E94C20666EE06
:1024F000D8018D919C910E94C206BE016F5F7F4FF3
:10250000C8010E949B0B0F900F908981882309F4CA
:102510007AC08A81882309F476C08DE893E09F937E
:102520008F930E94520566EEF801808191810E948E
:10253000C20668EED8018D919C910E94C20660E0AF
:10254000F801808191810E94C20668EED8018D91C8
:102550009C910E94C20663E0F801808191810E94F3
:10256000C20668EED8018D919C910E94C20662E07D
:10257000F801808191810E94C20668EED8018D9198
:102580009C910E94C20661E0F801808191810E94C5
:10259000C20666EED8018D919C910E94C20668EE3B
:1025A000F801808191810E94C20663E0D8018D917B
:1025B0009C910E94C20668EEF801808191810E9480
:1025C000C20661E0D8018D919C910E94C20668EE1E
:1025D000F801808191810E94C20662E0D8018D914C
:1025E0009C910E94C20668EEF801808191810E9450
:1025F000C20663E0D8018D919C910E94C20689E0D9
:10260000F801848781C086E893E09F938F930E94AE
:10261000520563EFD8018D919C910E94C20668EC2F
:10262000F801808191810E94C20663EFD8018D91EB
:102630009C910E94C20664E6F801808191810E940B
:10264000C20663EFD8018D919C910E94C20660E59D
:10265000F801808191810E94C206C8010E94B40CD9
:10266000292F30E00F900F902330310511F080E0DA
:1026700001C083E0D8011C968C938FE793E09F9371
:102680008F930E94520563EFF801808191810E942F
:10269000C20668ECD8018D919C910E94C20663EF3E
:1026A000F801808191810E94C20668ECD8018D9169
:1026B0009C910E94C20663EFF801808191810E9483
:1026C000C20660E5D8018D919C910E94C206C801A6
:1026D0000E94B40C292F30E00F900F902430310568
:1026E00011F080E001C084E0F801848781110EC000
:1026F00088E793E09F938F930E94520566EFD8017D
:102700008D919C910E94C2060F900F9064EFF8018A
:10271000808191810E94C206BE016F5F7F4FC80118
:102720000E949B0BD8011C968C91893049F0833014
:1027300051F0843059F0882361F083E291E00BC0BE
:102740008FE491E008C087E491E005C088E591E05E
:1027500002C081E691E09F938F938CE693E09F9374
:102760008F930E9452050F900F900F900F908BE067
:10277000F80180870E94782C9F938F9387E693E0DF
:102780009F938F930E9452050F900F900F900F9080
:10279000D8018D919C910E9466064C01019609F426
:1027A0001DC2F8018481843069F18114910421F003
:1027B000FFEF8F16910469F40E94D50B0E94E72168
:1027C0008FE593E09F938F930E9452050F900F9097
:1027D00005C2823069F0833081F0813009F0FEC19A
:1027E000682DC8010E943D0D8F3F09F0F7C112C04E
:1027F000682DC8010E94170EF7CF682DC8010E94EE
:10280000FA0EF2CFF801808191810E94A7066C0137
:10281000019629F48CE0D80118968C93DFC1F80159
:10282000808191810E94A7067C01019699F3D801CD
:102830001C968C91FE0131965F01853028F483301F
:1028400030F4882321F0DCC08930A1F0D9C0D80150
:102850001D969C911D97987F282D2770922B1D9671
:102860009C9384FE02C0DD24DA9485FEC4C0FF245C
:10287000FA94C1C0F8013585C40188749927883459
:10288000910509F0A9C0C1FEA7C0F0E38F229924E9
:10289000959487949594879420E3C222DD2454E094
:1028A000D594C7945A95E1F7C828D92842E0C416B0
:1028B000D104E1F183E0C816D10409F476C0CA94CA
:1028C000CD2809F07CC1E6FC17C0A7014870552748
:1028D0008E2D8F70E7FE07C0452B11F420E001C05C
:1028E00020EF822B0AC0452B11F420E001C020EF1D
:1028F000982F922B80E002C080E090E0E4FE05C0BB
:102900003860D8011D963C9303C0377FF8013587A6
:10291000D8011D962C911D97E5FE04C020611D96DF
:102920002C934FC12F7EF80125874BC1E0FE05C0D7
:102930003064D8011D963C9303C03F7BF801358776
:10294000D8011D968C911D97E1FE04C080681D96EC
:102950008C9303C08F77F8018587D8011D968C91E1
:102960001D97E2FE04C080621D968C9303C08F7D8C
:10297000F8018587D8011D968C911D97E3FE04C050
:1029800080641D968C9303C08F7BF8018587D801E6
:102990001D968C911D97E4FE04C080681D968C9353
:1029A0000EC18F77F80185870AC1C70124E095958C
:1029B00087952A95E1F7E7FE03C0806F90E003C09A
:1029C000982F9F7080E0387F2E2D2770E32EE22A0B
:1029D000D8011D96EC92F5C0387F882D8770382B72
:1029E000F801358784FE02C0DD24DA9485FE4DC0EF
:1029F000FF24FA944AC0833049F08430C9F045C0BE
:102A0000833079F4E12CF12CC12CD12CD8018D919B
:102A10009C910E94A7068F3FBFEF9B07B1F1982FB3
:102A200035C0843009F0CBC0E12CF12CC12CD12C65
:102A3000F801808191810E94A706AC018F3FFFEFD2
:102A40009F0719F183FD02C080E001C080EF942F41
:102A50009F70982BD8011D962C911D9744FF04C0A0
:102A600028601D962C9303C0277FF8012587D80185
:102A70001D962C911D9745FF04C020611D962C9337
:102A800005C02F7EF801258701C090E085E0D501C3
:102A90001D928A95E9F7F8018585898380E0F0E841
:102AA000CF16D1044CF4960141E8C4164FEFD4067A
:102AB00024F421E83FEF01C02FE72A83A0E8EA16BB
:102AC000F10454F49701B1E8EB16BFEFFB0614F4E0
:102AD00021E83FEF219501C021E82B83903811F0C8
:102AE000919501C09FE79C83803809F481E88D832C
:102AF000C5010E942A1F89811F928F938D81282FE3
:102B0000082E000C330B3F938F938C81282F082EB7
:102B1000000C330B3F938F938B81282F082E000CD2
:102B2000330B3F938F938A81282F082E000C330B91
:102B30003F938F9380E493E09F938F930E9452057D
:102B40000FB6F894DEBF0FBECDBF48C00E94E7218C
:102B5000D80118961C9242C0828185FF93CAD80181
:102B600018968C918B3009F08DCA84E094E09F9385
:102B70008F930E9452058CE0F80180870F900F9090
:102B800081CA8CEC93E09F938F930E9452050F9023
:102B90000F909ECB60EFF801808191810E94C20668
:102BA0008A3F910509F094CB63E0D8018D919C9107
:102BB0000E94C2068A3F910509F08ACBD4CB80E0FF
:102BC00090E025E0D5011D922A95E9F7F8012585C9
:102BD0002983E12CF12CC12CD12C65CF81E00F9001
:102BE0000F900F900F900F90DF91CF911F910F9149
:102BF000FF90EF90DF90CF90BF90AF909F908F901D
:102C0000089588EC91E00E94C60F8AEB91E00C9445
:102C1000C60FE8ECF1E08DE991E0918380831382A7
:102C200012821482158210861186128613861486EB
:102C300015860E94D50BEAEBF1E080E891E09183E4
:102C40008083138212821482158210861186128666
:102C50001386148615860C94D50B80910A0308956B
:102C6000CF93DF9300D01F92CDB7DEB72091180429
:102C7000243021F523E029839B838A8382E080939B
:102C8000E9008FEF9091E800815095FD06C095ED29
:102C90009A95F1F700008111F5CF8091E80085FF4A
:102CA0000DC040E050E063E070E0CE0101960E946C
:102CB000001B8091E8008E778093E8000F900F90C2
:102CC0000F90DF91CF910895CF93DF9300D01F92A3
:102CD000CDB7DEB720911804243061F519821A822D
:102CE0001B8222E029838138910520F080589109C8
:102CF0009B838A8382E08093E9008FEF9091E800C4
:102D0000815095FD06C095ED9A95F1F7000081116F
:102D1000F5CF8091E80085FF0DC040E050E063E012
:102D200070E0CE0101960E94001B8091E8008E7732
:102D30008093E8000F900F900F90DF91CF9108954E
:102D400020911804243051F522E02093E9002FEF60
:102D50003091E800215035FD06C035ED3A95F1F788
:102D600000002111F5CF2091E80025FF17C0209128
:102D70001001222341F021E02093F10040E050E0D7
:102D800065E070E004C040E050E063E070E00E9465
:102D9000001B8091E8008E778093E8000895CF9320
:102DA000DF9320911804243009F04AC0EC0180918F
:102DB00011018823E1F0809112018823C1F081E0A4
:102DC0008093E90081E8815049F09091E80095FDF9
:102DD00005C09AE29A95F1F700C0F5CF8091E8001E
:102DE00085FF2EC040E050E060E270E019C081E055
:102DF0008093E90081E8815059F09091E80095FDB9
:102E000007C0EFE3F1E03197F1F700C00000F3CF26
:102E10008091E80085FF14C040E050E068E070E079
:102E2000CE010E94001B8091E8008E778093E8001D
:102E300080E2FE01AAEEB2E001900D928A95E1F7E0
:102E4000DF91CF910895CF93C091E801C1110BC0DC
:102E50000E94842C643C79408105910520F081E03A
:102E60008093E801C1E08C2FCF910895FF920F93DA
:102E70001F93CF93DF93D82F0FB607FE83C08091A7
:102E80001804843081F08091030190E00196209134
:102E9000050130E0822393232091040130E0821762
:102EA000930709F0CDC00E942317811110C08091B3
:102EB000030190E001962091050130E082239323E5
:102EC0002091040130E08217930709F0B9C00E94F5
:102ED000782C8C01C091E900CF709091EC00892F83
:102EE000817090FD80E8C82B83E08093E90085E045
:102EF000F82E8091EB0085FD42C08091EB0080FFB1
:102F00003EC08091EE0087FF3AC08091040190910D
:102F10000301981709F457C09091E80095FF8EC0FF
:102F2000E0910101F0910201E80FF11D20818F5F16
:102F3000909105018923809304012093F1008091F1
:102F4000E80085FDE2CF8091E80080FFDECF809130
:102F5000E8008E778093E800F0920001D6CF809150
:102F6000030190E001962091050130E08223932334
:102F70002091040130E08217930709F44CC0CF7010
:102F8000C093E90040910301842F90E001962091C5
:102F9000050130E0822393232091040130E0821761
:102FA000930709F450C0E0910101F0910201E40F90
:102FB000F11DD083809103018F5F909105018923DA
:102FC0008093030140C08091E80085FF37C0D09313
:102FD000F10021E03091F3008091F20090E0932B1A
:102FE000892B91F08091E80080FF0EC08091E8006D
:102FF00085FF03C01092F100F9CF8091E8008E7731
:103000008093E800F0920001222309F4A8CFCF704A
:10301000C093E90018C080910001882309F4AFCF64
:103020000E94782C9C018017910711F4890161CFCF
:1030300090910001915090930001F8CF20E0CACF09
:1030400040910301B0CF80E0DF91CF911F910F91AC
:10305000FF90089580911704811104C00E946C1D97
:103060000C94C91D0895109217040895089542E222
:1030700061EC81E00E94791A42E061EC82E00E94FA
:10308000791A42E261EC83E00C94791A80911A0477
:10309000833009F453C030F4813071F0823009F488
:1030A000BAC008958A3009F4A6C08B3009F478C0FC
:1030B000893009F0C8C020C080911904813A09F014
:1030C000C2C08091E800877F8093E80080911D0452
:1030D00090911E04892B21F460E28AEE92E003C0F5
:1030E00060E080E090E070E00E944D1B8091E8007D
:1030F0008B778093E800089580911904813209F05C
:10310000A2C080911D0490911E04892B09F09BC0E0
:103110008091E800877F8093E8008091E80082FD3D
:1031200005C0809118048111F8CF8DC08091F10005
:1031300080930A038091E8008B7781C08091190405
:10314000813A09F080C080911D0490911E04892B62
:10315000A1F48091E800877F8093E8008091E800E7
:1031600080FFFCCF809111018093F1008091E800F5
:103170008E778093E8000E94AE1A80911D04909192
:103180001E04019709F05FC08091E800877F80935B
:10319000E8008091E80080FFFCCF809110014AC0D8
:1031A00080911904813209F04EC080911D049091E4
:1031B0001E04892B69F48091E800877F8093E800E2
:1031C0000E94AE1A80911B04809311010E94E72196
:1031D00080911D0490911E040197A9F58091E8004B
:1031E000877F8093E8000E94AE1A80911B04809331
:1031F00010010C94E72180911904813221F580910E
:10320000E800877F8093E8000E94AE1A80911C043A
:1032100080930B03089580911904813AA1F4809161
:10322000E800877F8093E8008091E80080FFFCCF72
:1032300080910B038093F1008091E8008E7780935A
:10324000E8000C94AE1A089580910A038093E90176
:1032500010920A030E94560C0C94E7210C94241936
:103260000E94242C80911604882329F00E94312C7E
:1032700081110C94631A08950E94462C8091E901F3
:1032800080930A0308950C943C1908950C944519F1
:10329000CF9384B7877F84BF0FB6F894A8958091A9
:1032A0006000886180936000109260000FBE90E023
:1032B00080E80FB6F89480936100909361000FBE90
:1032C00086E397E10E94E32B86E091E00E94D01E06
:1032D00083EF95E00E94B9040E943A0C0E948F1F70
:1032E0000E946C1D0E94C91D78940E94911F8091BC
:1032F0001804843029F00E94B51E0E944519F7CFAA
:1033000081EE95E00E94B9040E94461983ED95E094
:103310000E94B904C3E080911804853019F40E941A
:103320003019F9CF0E940D2C0E94951F2091E400C6
:103330003091E5008091E6019091E7012817390767
:1033400009F468C08091E4009091E5009093E70152
:103350008093E6010E942317882309F45BC08091C3
:103360001804843009F056C08091E9008F702091D4
:10337000EC00922F917020FD90E8892BC093E9001A
:103380009091EB0090FF43C09091EE0097FF3FC0FB
:103390009091040120910301291709F12091E8007F
:1033A00025FF1DC0E0910101F0910201E90FF11D1F
:1033B00030819F5F20910501922390930401309307
:1033C000F1009091E80095FDE3CF9091E80090FF27
:1033D000DFCF9091E8009E779093E800D9CF90914D
:1033E000F3002091F20030E0392B232B81F09091F3
:1033F000E80090FF0CC09091E80095FF03C0109288
:10340000F100F9CF9091E8009E779093E8008F70DB
:103410008093E9000E94B51E7ECF292F33272330E9
:103420003105C9F060F42130310581F022303105D9
:1034300009F041C08BE590E020E536E040C0213244
:103440003105E1F02232310531F135C082E190E001
:103450002BEA36E034C099278130910549F028F0F5
:10346000029749F5ECE0F6E005C0ECE4F6E002C0B6
:10347000E2E4F6E0849190E09F0121C063307105A1
:10348000D0F4660F771FFB01EE58FE4F208131818B
:1034900089E090E014C06330710568F4FB01EE0F21
:1034A000FF1FE459FE4F20813181FB01E759FE4F98
:1034B000808190E004C080E090E020E030E0FA01FC
:1034C00031832083089580E189BD82E189BD09B4FB
:1034D00000FEFDCF8091D8008F7D8093D800809131
:1034E000E00082608093E0008091E00081FDFCCFED
:1034F0000895982F973068F59093E900981739F060
:103500007091EC002091ED005091F00003C0242F49
:10351000762F50E021FD02C09F5FECCF3091EB0091
:103520003E7F3093EB003091ED003D7F3093ED0016
:103530003091EB0031603093EB007093EC002093FE
:10354000ED005093F0002091EE0027FDE5CF80E0E4
:1035500008958F708093E90081E0089580911904A7
:1035600087FF11C08091E80082FD05C0809118049A
:103570008111F8CF11C08091E8008B770BC080914A
:103580001804882349F08091E80080FFF8CF8091EB
:10359000E8008E778093E80008952091E400309150
:1035A000E50095E64091EC00842F817040FF23C038
:1035B0008091E80080FD1DC080911804882399F057
:1035C000853099F08091EB0085FD11C04091E400B9
:1035D0005091E5002417350729F3915011F09A0115
:1035E000E1CF84E0089582E0089583E0089581E0CA
:1035F000089580E008954091E80042FFDDCF0895EE
:10360000CF92DF92EF92FF920F931F93CF93DF93AE
:10361000EC018B017A010E94CD1A811135C0E114B1
:10362000F10439F0F70180819181081B190BC80F53
:10363000D91FC12CD12C0115110529F18091E80069
:1036400085FD18C08091E8008E778093E8000E9485
:10365000B51EE114F10449F0F70180819181C80E93
:10366000D91ED182C08285E00FC00E94CD1A882366
:1036700011F30AC089918093F10001501109FFEF05
:10368000CF1ADF0AD8CF80E0DF91CF911F910F9141
:10369000FF90EF90DF90CF90089520911F0430911C
:1036A00020042617370748F06115710539F4209179
:1036B000E8002E772093E80001C0B901FC0120E06A
:1036C0006115710579F1809118048823F1F1853035
:1036D000F1F18091E80083FD3CC08091E80082FD1B
:1036E0002EC08091E80080FFEBCF2091F300809105
:1036F000F20090E0922B6115710551F08830910530
:1037000038F421912093F100615071090196F3CFB3
:1037100021E0089709F020E08091E8008E778093FF
:10372000E800CECF2111CFCF0AC0809118048823A2
:1037300061F0853061F08091E80083FD0AC08091DE
:10374000E80082FFF2CF80E0089582E0089583E0F0
:10375000089581E0089520911F04309120042617D8
:10376000370748F06115710539F42091E8002E778C
:103770002093E80001C0B901FC0120E0611571054A
:1037800091F180911804882309F440C0853009F430
:103790003FC08091E80083FD3DC08091E80082FD3C
:1037A0002FC08091E80080FFE9CF2091F300809145
:1037B000F20090E0922B6115710559F08830910567
:1037C00040F424912093F1003196615071090196E3
:1037D000F2CF21E0089709F020E08091E8008E7791
:1037E0008093E800CBCF2111CCCF0AC08091180480
:1037F000882361F0853061F08091E80083FD0AC084
:103800008091E80082FFF2CF80E0089582E0089581
:1038100083E0089581E008951F93CF93DF93CDB7A0
:10382000DEB7AA970FB6F894DEBF0FBECDBFE9E1B1
:10383000F4E08091F100819324E0E132F207C9F7CE
:103840000E9446188091E80083FF2EC180911904E0
:1038500090911A04492F50E04A30510508F024C1D4
:10386000FA01E05CFE4F0C94DA30803821F08238A7
:1038700009F01AC108C0809115049091160499238B
:1038800089F082600FC080911D048F70873008F02E
:103890000BC18093E9008091EB0085FB882780F9BC
:1038A0001092E9009091E800977F9093E800809350
:1038B000F1001092F100D1C0282F2D7F09F0F4C043
:1038C000882319F0823061F0EFC080911B048130B1
:1038D00009F0EAC0933009F080E0809316042EC00E
:1038E00080911B0481112AC080911D048F702FEFDD
:1038F000280F263008F0D8C08093E9002091EB0013
:1039000020FF1CC0933021F48091EB00806214C032
:103910009091EB0090619093EB0021E030E0A901E1
:1039200002C0440F551F8A95E2F74093EA001092B7
:10393000EA008091EB0088608093EB001092E90030
:103940008091E800877F8093E8000E94AE1AACC0A7
:103950008111AAC010911B041F778091E300807829
:10396000812B8093E3008091E800877F8093E800BB
:103970000E94AE1A8091E80080FFFCCF8091E300A6
:1039800080688093E300111102C082E001C083E0EF
:103990008093180489C08058823008F085C08091D7
:1039A0001B0490911C048C3D53E0950779F583E04E
:1039B0008A838AE289834FB7F894DE01139620E068
:1039C0003EE051E2E32FF0E050935700E49120FFF6
:1039D00003C0E295EF703F5FEF708E2F90E0EA300A
:1039E00010F0C79601C0C0968D939D932F5F243130
:1039F00049F74FBF8091E800877F8093E8006AE233
:103A000070E0CE0101960E944D1B16C060911D040E
:103A100070911E04AE014F5F5F4F0E940D1ABC01F2
:103A2000892B09F441C09091E800977F9093E800BA
:103A300089819A810E94AB1B8091E8008B778093EB
:103A4000E80032C0803881F58091E800877F80935C
:103A5000E800809114048093F1008091E8008E7753
:103A600072CF811121C080911B0490911C04992771
:103A70000297D4F48091E800877F8093E8008091DA
:103A80001B04809314040E94AE1A809114048111C7
:103A900006C08091E30087FD02C081E001C084E0A0
:103AA000809318040E9437188091E80083FF0AC0B1
:103AB0008091E800877F8093E8008091EB0080622E
:103AC0008093EB00AA960FB6F894DEBF0FBECDBF71
:103AD000DF91CF911F9108950E94DA1D0E94E21D8F
:103AE000E0EEF0E0808181608083E8EDF0E08081AD
:103AF0008F77808319BCA7EDB0E08C918E7F8C937B
:103B000080818F7E80831092170408950F931F93F6
:103B1000CF93DF930E94DA1D0E94E21DC8EDD0E032
:103B200088818F77888388818068888388818F7D6A
:103B3000888319BC10921804109214041092160471
:103B40001092150400EE10E0F80180818B7F8083D5
:103B500088818160888342E060E080E00E94791A79
:103B6000E1EEF0E080818E7F8083E2EEF0E0808104
:103B700081608083808188608083F80180818E7F6E
:103B80008083888180618883DF91CF911F910F911D
:103B90000895E8EDF0E080818F7E8083E7EDF0E02E
:103BA00080818160808384E082BF81E080931704FC
:103BB0000C94861DE8EDF0E080818E7F808310926A
:103BC000E20008951092DA001092E10008951F9229
:103BD0000F920FB60F9211242F933F934F935F9341
:103BE0006F937F938F939F93AF93BF93EF93FF93C5
:103BF0008091E10082FF0BC08091E20082FF07C04C
:103C00008091E1008B7F8093E1000E94B41E80913F
:103C1000DA0080FF1FC08091D80080FF1BC0809118
:103C2000DA008E7F8093DA008091D90080FF0DC08A
:103C300080E189BD82E189BD09B400FEFDCF81E04C
:103C4000809318040E942A1805C019BC1092180409
:103C50000E9433188091E10080FF19C08091E2003A
:103C600080FF15C08091E2008E7F8093E2008091FA
:103C7000E20080618093E2008091D80080628093AE
:103C8000D80019BC85E0809318040E942E198091F9
:103C9000E10084FF30C08091E20084FF2CC080E10D
:103CA00089BD82E189BD09B400FEFDCF8091D800B5
:103CB0008F7D8093D8008091E1008F7E8093E1001A
:103CC0008091E2008F7E8093E2008091E20081602B
:103CD0008093E20080911404882311F084E007C0EF
:103CE0008091E30087FD02C081E001C083E0809302
:103CF00018040E9443198091E10083FF24C0809141
:103D0000E20083FF20C08091E100877F8093E10083
:103D100082E080931804109214048091E1008E7F59
:103D20008093E1008091E2008E7F8093E200809199
:103D3000E20080618093E20042E060E080E00E9467
:103D4000791A0E943618FF91EF91BF91AF919F9120
:103D50008F917F916F915F914F913F912F910F9034
:103D60000FBE0F901F9018950895CF93809118045F
:103D70008823A1F0C091E900CF709091EC00892FC9
:103D8000817090FD80E8C82B1092E9008091E800D6
:103D900083FD0E940C1CCF70C093E900CF91089561
:103DA00090931103809310030895E0911003F09114
:103DB0001103309721F00190F081E02D099480E00B
:103DC0000895EF92FF920F931F93CF93DF93E091AB
:103DD0001003F09111033097B1F18C010280F3814F
:103DE000E02D09958091060482FF2DC080FF04C05C
:103DF0008DEB97E00E94B904E80110E287EBE82E12
:103E000087E0F82E8091060480FF0BC088811F9206
:103E10008F93FF92EF920E9452050F900F900F9098
:103E20000F90115021961111EDCF8091060480FF63
:103E30000AC085EB97E0DF91CF911F910F91FF9022
:103E4000EF900C94B904DF91CF911F910F91FF90E7
:103E5000EF900895E0911003F0911103309721F055
:103E60000480F581E02D09940895CF93DF9320918C
:103E70000E0330910F032817390709F190930F03B0
:103E800080930E03E0911003F09111033097B9F085
:103E9000EC010680F781E02D09958091060482FFF0
:103EA0000EC080FF0CC0DF93CF9387EA97E09F930B
:103EB0008F930E9452050F900F900F900F90DF91FB
:103EC000CF910895CF93DF9320910C0330910D0390
:103ED0002817390709F190930D0380930C03E091A3
:103EE0001003F09111033097B9F0EC010084F185D3
:103EF000E02D09958091060482FF0EC080FF0CC062
:103F0000DF93CF9387E997E09F938F930E945205A9
:103F10000F900F900F900F90DF91CF9108950C9418
:103F200050200E946F2C0C94460C8F929F92AF925F
:103F3000BF92CF92DF92EF92FF920F931F93CF9396
:103F4000DF9300D000D01F92CDB7DEB70E940116DC
:103F500003E113E0F12C8F2D0E944D0C4C01F80170
:103F6000A080B180A826B926A114B10439F4F39435
:103F70000E5F1F4FF8E0FF12EECF39C080910604AC
:103F800081FD0E946420E12CCC24C394D12CC50176
:103F90008C219D21892B21F1E982FA8221E0C40143
:103FA0008C219D21892B09F420E02B830E94782C01
:103FB0008160782F9D838C8349815A816B818D81AB
:103FC0000E949A2049815A816B817C818D810E9457
:103FD0000F2CF801808191818C259D259183808310
:103FE000E394CC0CDD1CF0E1EF12D1CFC0CF8FEF0A
:103FF00089838A831B820E94782C8160782F9D831D
:104000008C8349815A816B818D810E949A200E9404
:104010000E2C0E94E42E0E94D51E90911203891747
:1040200059F10E94D51E809312039091060492FFCD
:104030000EC090FF0CC01F928F9388EC97E09F9367
:104040008F930E9452050F900F900F900F908091C8
:1040500012030F900F900F900F900F90DF91CF9160
:104060001F910F91FF90EF90DF90CF90BF90AF9096
:104070009F908F900C94202C0F900F900F900F908A
:104080000F90DF91CF911F910F91FF90EF90DF90F4
:10409000CF90BF90AF909F908F9008950C94820C1A
:1040A0000895CF93C62F0E944D0C21E030E002C04E
:1040B000220F331FCA95E2F72823392381E0232BEF
:1040C00009F480E0CF910895EF92FF920F931F9330
:1040D000CF93DF938FED97E00E94B904C0E0D0E06A
:1040E00080E2E82E81E0F82E03ED17E08C2F0E948D
:1040F0004D0C0E94FA2BFF92EF929F938F93DF93C8
:10410000CF931F930F930E94520521968DB79EB7B0
:1041100008960FB6F8949EBF0FBE8DBFC830D1056C
:1041200029F7DF91CF911F910F91FF90EF900895A4
:1041300008950895CF93DF93CDB7DEB72B970FB6D1
:10414000F894DEBF0FBECDBF942F4F83252F588725
:1041500069877A878B874A855B85452B31F02F3FAE
:1041600031F481E09F3F19F403C081E001C080E099
:1041700080FD07C04F81588569857A858B850E94AF
:104180000F2CDE01119686E0FD0111928A95E9F768
:1041900085E0FE01379601900D928A95E1F74981FD
:1041A0005A816B817C818D819E810E9400282B9693
:1041B0000FB6F894DEBF0FBECDBFDF91CF9108954B
:1041C000882309F4BBC09CEF980F913A18F40E9421
:1041D000DE2A0DC090E2980F983058F4877091E075
:1041E00001C0990F8A95EAF7892F0E94832B0C94BE
:1041F000BD2B9BE5980F933070F4853A29F0863AF1
:1042000031F083E890E005C081E890E002C082E8E8
:1042100090E00C94351F98E5980F973108F08EC008
:10422000883A09F445C0893A09F445C08A3A09F444
:1042300045C08B3A09F445C08C3A09F445C08D3A23
:1042400009F445C08E3A09F445C08F3A09F445C0D7
:10425000813B09F445C0803B09F445C0823B09F429
:1042600045C0833B09F445C0843B09F445C0853B08
:1042700009F445C0863B09F445C0873B09F445C0B5
:10428000883B09F445C0893B09F445C08A3B09F4E1
:1042900045C08B3B09F445C08C3B09F445C08D3BC0
:1042A00009F445C08E3B09F445C080E090E044C06D
:1042B00082EE90E041C089EE90E03EC08AEE90E050
:1042C0003BC085EB90E038C086EB90E035C083EBD7
:1042D00090E032C084EB90E02FC087EB90E02CC0E0
:1042E0008CEC90E029C08DEC90E026C083E891E052
:1042F00023C08AE891E020C082E991E01DC084E9F2
:1043000091E01AC081E292E017C083E292E014C00B
:1043100084E292E011C085E292E00EC086E292E073
:104320000BC087E292E008C08AE292E005C08FE607
:1043300090E002C080E790E00C94621F089588230B
:1043400029F19CEF980F913A18F40E942E2B0DC082
:1043500090E2980F983058F4877091E001C0990F5F
:104360008A95EAF7892F0E94892B0C94BD2B9BE537
:10437000980F933020F480E090E00C94351F885A19
:10438000873120F480E090E00C94621F0895882328
:1043900021F00E94832B0C94BD2B0895882321F0DB
:1043A0000E94892B0C94BD2B08950E94A32B0E9480
:1043B000722B0E94BD2B0E94892F0E94572E80E0F5
:1043C00090E00E94351F80E090E00C94621F0E94F4
:1043D000932B0C94D521CF92DF92EF92FF920F9303
:1043E0001F93CF93DF9300D000D01F92CDB7DEB7DD
:1043F0006C010E94222C811118C385E0F601DE01B8
:10440000119601900D928A95E1F7F6014081518154
:10441000238134812115310531F05F3F31F481E092
:104420004F3F19F403C081E001C080E080FDFDC270
:10443000F601F280E580E2948FE0E82249835A8316
:10444000FB82722F3D832C836F2D8D810E945A2A0F
:104450008C010E94592A0E945329E12FE295EF70A6
:104460008E2F90E0FC01E65BFE4F0C94DA30812F3A
:10447000807F1F70882311F01295107FFF20B9F004
:10448000112329F0812F0E94962B0E94BD2B802F93
:104490000F900F900F900F900F90DF91CF911F9181
:1044A0000F91FF90EF90DF90CF900C94E020802F41
:1044B0000E949F21112309F4B8C2812F0E949C2BD6
:1044C0000F900F900F900F900F90DF91CF911F9151
:1044D0000F91FF90EF90DF90CF900C94BD2B812F28
:1044E000807F1F70803211F01295107F002319F029
:1044F000013009F12BC0FF20A9F0EE2059F1F1E0C5
:10450000812FEF1228C00F900F900F900F900F90F7
:10451000DF91CF911F910F91FF90EF90DF90CF909F
:104520000C94A62BEE2021F021E0E21609F47DC2C6
:104530000E94A92B4DC0FF20E9F085E08E1508F4FC
:1045400074C20E94802B812329F042C0FF20F1F128
:10455000E11015C0812F0F900F900F900F900F90CA
:10456000DF91CF911F910F91FF90EF90DF90CF904F
:104570000C94C72194E09E1508F457C229C0F60197
:10458000858180FF13C08F708583E4CF003F09F4DD
:1045900089C108F055C180E4800F803208F459C108
:1045A000FF2009F4EAC1EE2009F49AC1802F0E948D
:1045B000E020093309F0DAC1FFEF21EE84E0F15089
:1045C00020408040E1F700C000002FC2E110D7C1B9
:1045D000812F59C1812F86958695837019F081307E
:1045E000B9F023C2FF2019F0C801937002C080E027
:1045F00090E00F900F900F900F900F90DF91CF9160
:104600001F910F91FF90EF90DF90CF900C94351F8A
:10461000FF2019F0C801937002C080E090E00F9075
:104620000F900F900F900F90DF91CF911F910F91EE
:10463000FF90EF90DF90CF900C94621F802FFF20AF
:1046400019F00E946A2D02C00E94D22D0F900F9087
:104650000F900F900F90DF91CF911F910F91FF90CE
:10466000EF90DF90CF900C94572E812F837009F03C
:1046700070C0F110DAC1202F229526952770220FE5
:10468000220F602F6F70862F90E0A0E0B0E06C01E9
:104690007D01022E04C0CC0CDD1CEE1CFF1C0A9414
:1046A000D2F704FF12C08FE090E0A0E0B0E004C0B9
:1046B000880F991FAA1FBB1F2A95D2F7BC01CD01F5
:1046C000609570958095909503C060E070E0CB0197
:1046D0001695169513701230B1F040F56C297D29AE
:1046E0008E299F29113031F10F900F900F900F906C
:1046F0000F90DF91CF911F910F91FF90EF90DF907E
:10470000CF900C946E296C297D298E299F290F90BA
:104710000F900F900F900F90DF91CF911F910F91FD
:10472000FF90EF90DF90CF900C9488290E946E2923
:10473000C701B6010F900F900F900F900F90DF916F
:10474000CF911F910F91FF90EF90DF90CF900C943D
:104750005429FF2019F0812F817001C0869588238C
:1047600009F463C1202F229526952770220F220F6E
:10477000602F6F70862F90E0A0E0B0E06C017D01AB
:10478000022E04C0CC0CDD1CEE1CFF1C0A94D2F7D8
:1047900004FF12C08FE090E0A0E0B0E004C0880FFA
:1047A000991FAA1FBB1F2A95D2F7BC01CD016095A6
:1047B00070958095909503C060E070E0CB011695F0
:1047C000169513701230B1F040F56C297D298E29B1
:1047D0009F29113031F10F900F900F900F900F9093
:1047E000DF91CF911F910F91FF90EF90DF90CF90CD
:1047F0000C94352A6C297D298E299F290F900F90C2
:104800000F900F900F90DF91CF911F910F91FF901C
:10481000EF90DF90CF900C94472A0E94352AC70171
:10482000B6010F900F900F900F900F90DF91CF91E6
:104830001F910F91FF90EF90DF90CF900C94232A5F
:10484000023F09F45EC008F449C0033F09F46CC09C
:10485000A7CE902F9071E92E812F8F71FF2051F0FC
:104860000E94BC29802FEE2019F08295807F73CEA4
:104870008F7071CE0E94DD29802FEE2019F0829575
:10488000807F01C08F700F900F900F900F900F904E
:10489000DF91CF911F910F91FF90EF90DF90CF901C
:1048A0000C94CE21FF20A9F0E4E0EE1508F4BDC081
:1048B000812F8F710F900F900F900F900F90DF91BD
:1048C000CF911F910F91FF90EF90DF90CF900C94BC
:1048D000022AF5E0FE1508F4A8C0EACFFF2099F0FF
:1048E000812F8F710F900F900F900F900F90DF918D
:1048F000CF911F910F91FF90EF90DF90CF900C948C
:10490000BC29FF2069F3812F8F710F900F900F90BA
:104910000F900F90DF91CF911F910F91FF90EF902B
:10492000DF90CF900C94DD29FF2089F0812F8F71CB
:104930000F900F900F900F900F90DF91CF911F91DC
:104940000F91FF90EF90DF90CF900C94A7290F90DC
:104950000F900F900F900F90DF91CF911F910F91BB
:10496000FF90EF90DF90CF900C94A229033509F4CB
:1049700023CE073409F059C01FCEEE2021F2802F3C
:104980000F900F900F900F900F90DF91CF911F918C
:104990000F91FF90EF90DF90CF900C949F21412FCB
:1049A0004F70602FC6010E94E42C0F900F900F9063
:1049B0000F900F90DF91CF911F910F91FF90EF908B
:1049C000DF90CF900C94AE2801112FC0FF2069F129
:1049D0000E94E7212FEF80E792E021508040904035
:1049E000E1F700C000000F900F900F900F900F9014
:1049F000DF91CF911F910F91FF90EF90DF90CF90BB
:104A00000C94C52C412F4F70602FC6010F900F9052
:104A10000F900F900F90DF91CF911F910F91FF900A
:104A2000EF90DF90CF900C94E72C0F900F900F90A9
:104A30000F900F90DF91CF911F910F91FF90EF900A
:104A4000DF90CF9008951F93CF93DF9300D000D0D5
:104A50001F92CDB7DEB7942F4983252F5A836B83DE
:104A60007C838D834C815D81452B31F02F3F31F468
:104A700081E09F3F19F403C081E001C080E0182F5E
:104A8000117080FD24C049815A816B817C818D81A8
:104A90000E945A2A292F22952F702C3030F42A3068
:104AA00048F42250223068F013C02C3061F02F30CF
:104AB00051F00EC0803C28F0803E50F0815F833082
:104AC00038F011E005C093FB112710F901C010E088
:104AD000812F0F900F900F900F900F90DF91CF913B
:104AE0001F910895CF93DF9300D000D01F92CDB7D0
:104AF000DEB70F900F900F900F900F90DF91CF9136
:104B00000895CF93DF9300D000D000D0CDB7DEB7AB
:104B100026960FB6F894DEBF0FBECDBFDF91CF91C2
:104B200008951F93CF93DF93C091230316E08091E4
:104B30002403C81799F0D0E01C9FF0011D9FF00DD1
:104B40001124EB5DFC4F408151816281738184812E
:104B500095810E9481252196C770E9CFDF91CF9181
:104B60001F9108954091550350915603609157034A
:104B7000709158038091590390915A030C948125A8
:104B80000F931F93CF93DF9380915A0382958F7079
:104B900009F05DC080915703882309F458C08091C3
:104BA0002303109124036091550370915603C09123
:104BB0005803D091590391E06F3F09F090E0292FFD
:104BC00006E0811709F443C0209721F07F3F21F0D0
:104BD00030E003C031E001C0322F90E030FD34C03E
:104BE000089FF001099FF00D1124DF01AB5DBC4F60
:104BF00011963C911197371327C03C91361324C06E
:104C000012963C91129731111FC013964D915C91F1
:104C100014974C1B5D0B483C5105B0F480915A032E
:104C20008F70806180935A03E65DFC4F80818F70A6
:104C30008061808385E593E00E94EB21DF91CF9135
:104C40001F910F910C94912501968770BACFDF9137
:104C5000CF911F910F9108959F92AF92BF92CF92E3
:104C6000DF92EF92FF920F931F93CF93DF93CDB715
:104C7000DEB761970FB6F894DEBF0FBECDBF8C01D3
:104C800085E0F801DE011D9601900D928A95E1F70D
:104C9000F80140815181F280C380D4809091550306
:104CA0006091560320915803309159032115310525
:104CB00031F06F3F31F481E09F3F19F403C081E090
:104CC00001C080E0F82FF1709F2E80FD52C185E574
:104CD000A82E83E0B82EE0905703F601E21BF30BF9
:104CE000EE2009F4E8C080915A03E83CF10508F091
:104CF000A4C0282F207F09F053C0561313C04913B6
:104D000011C0EF2CF1100EC08F70806180935A0398
:104D10000E94B225C5010E94EB2180915A03F8013F
:104D200085835BC1C114D10431F05F3F31F481E070
:104D30004F3F19F403C081E001C080E080FD03C053
:104D400081E08F2502C080E090E0F82FF170EF2E17
:104D500080FF1CC0809123032091240336E082173A
:104D600009F418C190E0389FF001399FF00D11242B
:104D7000EB5DFC4F6181561306C06081461303C092
:104D80006281F61203C001968770E9CFEF2CFF20F5
:104D900009F423C180915A03816080935A0362C051
:104DA000561306C0491304C0F11002C0F801A7C091
:104DB0004D875E87FF867C2DD98AC88A6F2D8989A9
:104DC0000E942325882399F1FF2089F120915A031D
:104DD000822F82958F7090E0029774F08091550336
:104DE0009091560398878F831986DB86CA862C8715
:104DF000CE0107960E94EB2186E0F801A5E5B3E01D
:104E000001900D928A95E1F70E94C0250E94B2257B
:104E100011C0561749F14D875E87FF867C2DD98AD0
:104E2000C88A6F2D89890E94232581112CC0C80151
:104E30000E94EB21EE24E394D0C0282F207F49F775
:104E40007C2DD98AC88A6F2D89890E94722585E5B3
:104E500093E00E94EB2186E0F50111928A95E9F733
:104E60000E94B225E12CB9C04913D5CFF110D3CFA0
:104E7000F8018583C8010E94EB2186E0F5011192BB
:104E80008A95E9F7AAC0FF2091F220915A03822F58
:104E900082958F7090E002970CF4AECF809155030D
:104EA000909156039A8389831B82DD82CC822E8364
:104EB000CE0101969FCFE83CF10508F04BC0EF2CE6
:104EC000FF2009F4B4CF561330C049132EC02091EF
:104ED0005A0320FD21C0822F82958F70482F50E009
:104EE00041155105C9F0F80125834F30510541F0B6
:104EF0008F5F982F9295907F822F8F70892B85835B
:104F0000C8010E94EB2186E0F801A5E5B3E001901D
:104F10000D928A95E1F72AC086E0F801A5E5B3E095
:104F200001900D928A95E1F758C04D875E87FF8604
:104F30007C2DD98AC88A6F2D89890E9423258111E9
:104F40005BCF80915A03816080935A03C8010E940D
:104F5000EB2143C07C2DD98AC88A6F2D89890E9494
:104F6000722586E0F50111928A95E9F70E94B22533
:104F700034C0FF2009F45BCF4D875E87FF867C2D10
:104F8000D98AC88A6F2D89890E942325882309F42C
:104F90004ECF32CF7C2DD98AC88A6F2D89890E9445
:104FA0005A2A292F22952F70223028F49F7039F029
:104FB000811105C00BC0243028F49F7049F4805E35
:104FC000883020F0C8010E94EB219E2CE92C05C0FE
:104FD000F8019581907F99F7F9CF8E2D61960FB6E4
:104FE000F894DEBF0FBECDBFDF91CF911F910F911F
:104FF000FF90EF90DF90CF90BF90AF909F9008957B
:105000001F93CF93DF93CDB7DEB72C970FB6F894ED
:10501000DEBF0FBECDBF4F83588769877A878B87E6
:105020009C87CE0107960E942C268823D1F09F8171
:1050300088852A853B85232B31F08F3F31F481E031
:105040009F3F19F403C081E001C080E080FD47C0AC
:105050004F81588569857A858B859C850E9481253D
:105060003EC086E0FE013796DE01119601900D925A
:105070008A95E1F7FF81E8856A857B856115710571
:1050800031F0EF3F31F481E0FF3F19F403C081E0DC
:1050900001C080E080FD23C02091240330E0C901DD
:1050A0000196877099274091230350E08417950754
:1050B000F1F1F983EA837D836C8396E0929FD001BE
:1050C000939FB00D1124AB5DBC4FFE013196019052
:1050D0000D929A95E1F7809324030E94912516E0A2
:1050E0008091230390912403891771F1189FC001C7
:1050F00011248B5D9C4F0E942C26882329F1E0917E
:1051000023031E9FF0011124EB5DFC4F4081518170
:1051100062817381848195810E948125809123031E
:1051200090E001968770992780932303D9CF0E943E
:10513000E7211092240310922303E5E5F3E086E0D3
:10514000DF011D928A95E9F72C960FB6F894DEBF21
:105150000FBECDBFDF91CF911F910895DF92EF92E7
:10516000FF920F931F93CF93DF93FC01892B09F4D8
:1051700088C0E12CF12CDD24D394EF012196849199
:10518000853709F460C058F4843708F04EC0843085
:1051900008F068C08130D1F0823071F172C0883778
:1051A00009F45BC050F4863709F453C0873709F01F
:1051B00068C08E2D0E94902B52C09CE7980F9037AC
:1051C00008F05FC08F770E949F214EC08F010E5F55
:1051D0001F4FFE01849190E2980F983050F4877031
:1051E000FD2D01C0FF0F8A95EAF78F2F0E94962BA5
:1051F00015C00E94E02014C08F010E5F1F4FFE01FA
:10520000849190E2980F983068F48770FD2D01C06A
:10521000FF0F8A95EAF78F2F0E949C2B0E94BD2BCF
:10522000E80122C00E949F21FBCFCF010296FE0120
:10523000C491CC2361F0EFE9FFE03197F1F700C0B2
:105240000000C150F6CFCF010296FE01F490EC01B0
:105250000BC00E94802BE82E07C00E94932B0E9457
:10526000BD2B02C00E94E0208F2D882341F0EFE982
:10527000FFE03197F1F700C000008150F6CFFE014A
:105280007CCFDF91CF911F910F91FF90EF90DF9036
:1052900008956093DB037093DC038093DD039093A8
:1052A000DE030C941F2C08950F931F930091DF03CE
:1052B0001091E0032091E1033091E203602B712B08
:1052C000822B932B6093DF037093E0038093E103C1
:1052D0009093E2031F910F910C941E2C0F931F9338
:1052E0000091DF031091E0032091E1033091E2038C
:1052F00060237123822393236093DF037093E00381
:105300008093E1039093E2031F910F910C941E2C64
:105310000F931F930091DF031091E0032091E103AD
:105320003091E20360277127822793276093DF0380
:105330007093E0038093E1039093E2031F910F9138
:105340000C941E2C60E070E0CB010C9449290F9363
:105350001F9341E050E060E070E08A019B0104C0CF
:10536000000F111F221F331F8A95D2F7C901B80100
:105370001F910F910C9449290F931F9341E050E026
:1053800060E070E004C0440F551F661F771F8A95C8
:10539000D2F78091DB039091DC03A091DD03B09103
:1053A000DE038A019B01082B192B2A2B3B2BC901F9
:1053B000B8011F910F910C9449290F931F9341E05D
:1053C00050E060E070E004C0440F551F661F771F77
:1053D0008A95D2F740955095609570958091DB0342
:1053E0009091DC03A091DD03B091DE038A019B0163
:1053F000082319232A233B23C901B8011F910F91C8
:105400000C9449290F931F9341E050E060E070E055
:1054100004C0440F551F661F771F8A95D2F78091ED
:10542000DB039091DC03A091DD03B091DE038A01E0
:105430009B01082719272A273B27C901B8011F917B
:105440000F910C9449290F931F930091DB03109146
:10545000DC032091DD033091DE03602B712B822B66
:10546000932B1F910F910C9449290F931F93009137
:10547000DB031091DC032091DD033091DE03602318
:105480007123822393231F910F910C9449290F9329
:105490001F930091DB031091DC032091DD03309119
:1054A000DE0360277127822793271F910F910C94A9
:1054B000492908958F929F92AF92BF92DF92EF9207
:1054C000FF920F931F93CF93DF9300D000D01F92D2
:1054D000CDB7DEB76B837C838D838A018C819D8100
:1054E000892B31F01F3F31F481E04F3F19F403C0A5
:1054F00081E001C080E080FF03C080E090E04DC00B
:105500008B818823D1F18090DB039090DC03A09005
:10551000DD03B090DE038091DF039091E003A09162
:10552000E103B091E203882A992AAA2ABB2A8FE1D3
:10553000E82EF12CD501C4010E2C04C0B695A79518
:10554000979587950A94D2F780FD06C081E0E81A06
:10555000F10880F7D12C07C0DE2CB8018E2D0E94F7
:10556000580C019799F380E1189FF0011124E55A36
:10557000FC4FE00FF11DD08209C080E1189FF001BF
:105580001124E55AFC4FE00FF11DD08009831A83E6
:1055900069817A818D2D0E94580C0F900F900F9089
:1055A0000F900F90DF91CF911F910F91FF90EF908F
:1055B000DF90BF90AF909F908F90089590911101D0
:1055C000992379F190911201992359F1982F969589
:1055D000969596959F31A1F0E0911301F0911401F9
:1055E000E90FF11D877021E030E0A90102C0440FEE
:1055F000551F8A95E2F7CA019181892B818308950D
:105600009091060490FF29C01F928F9382E198E049
:105610009F938F930E9452050F900F900F900F90C1
:1056200008952091130130911401F90132969FEFF2
:1056300040E05191851789F09F3F19F4511101C045
:10564000942F4F5F4E31A9F79F3F39F0F901E90FD1
:10565000F11D97FDFA9582830895089590911101A7
:10566000992381F190911201992361F1982F9695D8
:10567000969596959F31A9F0E0911301F091140150
:10568000E90FF11D877021E030E0A90102C0440F4D
:10569000551F8A95E2F7CA018095918189238183FC
:1056A00008959091060490FF1CC01F928F9384EF81
:1056B00097E09F938F930E9452050F900F900F9049
:1056C0000F900895E0911301F09114019F01225E63
:1056D0003F4F9281891301C012823196E217F3077E
:1056E000C1F7089581E090E0E0911301F091140179
:1056F000E80FF91F1082019680329105A9F70895ED
:1057000080910504089590910504892B80930504E8
:105710000895809590910504892380930504089548
:10572000809305040895109205040895909104044F
:10573000892B809304040895809590910404892313
:105740008093040408951092040408958093E30361
:1057500008951092E303089580911301909114012C
:10576000FC0131969C01205E3F4F80E091919111A8
:105770008F5FE217F307D1F70895E0911301F091DD
:105780001401809105048083E0911301F0911401CC
:10579000908180910404892B80838091E303882386
:1057A00061F0E0911301F09114019081892B8083C5
:1057B0000E94AC2B81111092E30380911301909110
:1057C00014010C94E11E90937F0180937E01089553
:1057D0008295982F937344E0949F900111248C7CC0
:1057E00086958695282B822F8575880F2A7A26958F
:1057F000822B0895CF93DF93D92F0E94E82BC82FD7
:105800008D2F0E94E82B2C2F30E0322F2227A90168
:10581000482BCA01DF91CF91089508950895CF9341
:10582000DF9300D000D01F92CDB7DEB70F900F905E
:105830000F900F900F90DF91CF91089508950895E4
:105840000C944E2080E0089583B7817F8C6083BFE5
:1058500083B7816083BF7894889583B78E7F83BF39
:105860000895CF930E9498200E9401160E949920CB
:10587000C0E08C2F0E944D0C892B29F4CF5FC830DB
:10588000C1F780E001C081E0CF9108950E94560CDD
:105890000C94E7211F920F920FB60F9211248F9351
:1058A0009F93AF93BF938091070490910804A091B8
:1058B0000904B0910A044196A11DB11D809307040B
:1058C00090930804A0930904B0930A04BF91AF9188
:1058D0009F918F910F900FBE0F901F90189582E0AF
:1058E00084BD93E095BD9AEF97BD80936E000895B7
:1058F0002FB7F8948091070490910804A0910904AF
:10590000B0910A042FBF08952FB7F894609107044F
:10591000709108048091090490910A042FBF0895A2
:105920009C014FB7F8948091070490910804A091CE
:105930000904B0910A044FBF821B930B0895789419
:105940001F920F920FB60F9211248F939F93AF93D4
:10595000BF938091070490910804A0910904B0912D
:105960000A040196A11DB11D8093070490930804B9
:10597000A0930904B0930A04BF91AF919F918F91B6
:105980000F900FBE0F901F9018950E946C1DF894F9
:1059900087E797E7909301088093000887E090EBF2
:1059A000DC018093210490932204A0932304B093FC
:1059B00024049CE088E10FB6F894A89580936000D9
:1059C0000FBE90936000FFCF80E090E008950895AF
:1059D00080910D0480FF0BC06091180185E0689FE5
:1059E000B001112475956795759567952BC081FF5A
:1059F00009C06091180185E0689FB0011124759578
:105A0000679520C082FF07C06091180185E0689FFC
:105A1000B001112417C090910E049923D1F0609128
:105A20001701961788F72091180185E0289F9001AB
:105A30001124929FA001939F500D112470E0CA0180
:105A40000E94C6306038710540F46115710519F483
:105A500006C065E070E0862F08958FE7089581E025
:105A6000089580910D0480FF08C06091160170E0D8
:105A7000759567957595679521C081FF06C0609102
:105A8000160170E07595679519C082FF04C060919A
:105A9000160170E010C090910E04992399F0609166
:105AA00015019617A0F780911601899FC001112456
:105AB00070E00E94C6306038710540F461157105D0
:105AC00019F406C061E070E0862F08958FE708950D
:105AD00081E00895803F21F40E94E82C819504C064
:105AE000813F29F40E94E82C809311040895823F9D
:105AF00021F40E94E82C819504C0833F29F40E9480
:105B0000E82C809310040895893F19F40E94312DE8
:105B100005C08A3F31F40E94312D81958093120493
:105B200008958B3F21F40E94312D819504C08C3F54
:105B300029F40E94312D809313040895843F21F4A9
:105B400080910F04816017C0853F21F480910F047C
:105B5000826011C0863F21F480910F0484600BC0E5
:105B6000873F21F480910F04886005C0883F31F49D
:105B700080910F04806180930F0408958D3F21F47C
:105B800080910D0481600BC08E3F21F480910D0443
:105B9000826005C08F3F29F480910D04846080935A
:105BA0000D040895803F39F48091110487FF6CC083
:105BB0001092110469C0813F29F4809111041816D4
:105BC000BCF362C090911004823F29F497FF5CC03F
:105BD0001092100459C0833F19F41916CCF354C025
:105BE000893F41F48091120418160CF04DC01092B8
:105BF00012044AC08A3F29F48091120487FF44C0EE
:105C0000F6CF8B3F39F48091130487FF3DC010928B
:105C100013043AC08C3F29F4809113041816BCF386
:105C200033C0843F21F480910F048E7F17C0853FDD
:105C300021F480910F048D7F11C0863F21F4809163
:105C40000F048B7F0BC0873F21F480910F04877F67
:105C500005C0883F31F480910F048F7E80930F043C
:105C600013C08D3F21F480910D048E7F0BC08E3FB9
:105C700021F480910D048D7F05C08F3F29F4809120
:105C80000D048B7F80930D048091100481110EC050
:105C90008091110481110AC080911204811106C003
:105CA00080911304811102C010920E040895809116
:105CB000060483FF7EC087E598E00E94B9048091C6
:105CC0000F041F928F9382E598E09F938F930E9419
:105CD000520580E598E00E94B90480911004282FB5
:105CE000082E000C330B3F938F938DE498E09F9325
:105CF0008F930E9452058BE498E00E94B904809132
:105D00001104282F082E000C330B3F938F9388E447
:105D100098E09F938F930E94520586E498E00E943A
:105D2000B90480911204282F082E000C330B3F93E6
:105D30008F9383E498E09F938F930E94520581E4B0
:105D400098E00E94B90480911304282F082E000CBB
:105D5000330B3F938F938EE398E09F938F930E9432
:105D600052058BE398E00E94B90480910E041F92C3
:105D70008F9388E398E09F938F930E94520586E368
:105D800098E00E94B90480910D041F928F9383E3E1
:105D900098E09F938F930E94520580E398E00E94C1
:105DA000B9048DB79EB74C960FB6F8949EBF0FBE40
:105DB0008DBF8FE094E00E942A1F0E94782C909360
:105DC0000C0480930B0408951F93CF93DF9380916D
:105DD0000B0490910C040E94902CAC0190910E0445
:105DE000992321F02091190130E006C020911A0179
:105DF0008AE0289F900111244217530708F485C0B8
:105E000080911004C0911104D091120410911304D8
:105E1000811107C0C11175C0D11173C0111171C0BA
:105E200074C09F3F19F09F5F90930E04181624F4DE
:105E30000E94E82C809310048091100487FF05C015
:105E40000E94E82C8195809310041C1624F40E9473
:105E5000E82C809311048091110487FF05C00E94F3
:105E6000E82C81958093110460911004662331F130
:105E7000C0911104CC2311F1062E000C770B880B76
:105E8000990B0E94CD2F23E333E343E35FE30E94AA
:105E900031300E94952F609310046C2FCC0F770B3C
:105EA000880B990B0E94CD2F23E333E343E35FE399
:105EB0000E9431300E94952F609311041D1624F426
:105EC0000E94312D809312048091120487FF05C037
:105ED0000E94312D819580931204111624F40E94A2
:105EE000312D809313048091130487FF05C00E9415
:105EF000312D819580931304DF91CF911F910C94E4
:105F0000572E9F3F09F08FCFA0CFDF91CF911F91E8
:105F10000895EFE0F4E085E0DF011D928A95E9F74E
:105F200010920E0410920D0408950E949C2F689404
:105F3000B1110C942B3008950E94103088F09F57B7
:105F400098F0B92F9927B751B0F0E1F0660F771F9D
:105F5000881F991F1AF0BA95C9F714C0B13091F093
:105F60000E942A30B1E008950C942A30672F782FD0
:105F70008827B85F39F0B93FCCF386957795679558
:105F8000B395D9F73EF490958095709561957F4FC4
:105F90008F4F9F4F0895E89409C097FB3EF490956A
:105FA0008095709561957F4F8F4F9F4F9923A9F0F2
:105FB000F92F96E9BB279395F69587957795679581
:105FC000B795F111F8CFFAF4BB0F11F460FF1BC0C5
:105FD0006F5F7F4F8F4F9F4F16C0882311F096E958
:105FE00011C0772321F09EE8872F762F05C0662306
:105FF00071F096E8862F70E060E02AF09A95660FBF
:10600000771F881FDAF7880F9695879597F9089577
:1060100057FD9058440F551F59F05F3F71F0479559
:10602000880F97FB991F61F09F3F79F0879508953E
:10603000121613061406551FF2CF4695F1DF08C05D
:10604000161617061806991FF1CF8695710561057A
:1060500008940895E894BB2766277727CB0197F922
:1060600008950E9444300C94B5300E94A73038F057
:106070000E94AE3020F0952311F00C949E300C94C9
:10608000A43011240C942B300E94083070F3959F9B
:10609000C1F3950F50E0551F629FF001729FBB271F
:1060A000F00DB11D639FAA27F00DB11DAA1F649FBB
:1060B0006627B00DA11D661F829F2227B00DA11D6E
:1060C000621F739FB00DA11D621F839FA00D611DF4
:1060D000221F749F3327A00D611D231F849F600D15
:1060E000211D822F762F6A2F11249F5750409AF03E
:1060F000F1F088234AF0EE0FFF1FBB1F661F771FCA
:10610000881F91505040A9F79E3F510580F00C9494
:106110009E300C942B305F3FE4F3983ED4F3869589
:1061200077956795B795F795E7959F5FC1F7FE2B34
:10613000880F911D9695879597F9089597F99F6710
:1061400080E870E060E008959FEF80EC08950024FF
:106150000A941616170618060906089500240A94CC
:1061600012161306140605060895092E0394000C52
:1061700011F4882352F0BB0F40F4BF2B11F460FFE1
:1061800004C06F5F7F4F8F4F9F4F089597FB072E7F
:1061900016F4009407D077FD09D00E94E03007FC88
:1061A00005D03EF4909581959F4F08957095619527
:1061B0007F4F0895EE0FFF1F0590F491E02D099495
:1061C000AA1BBB1B51E107C0AA1FBB1FA617B7071D
:1061D00010F0A61BB70B881F991F5A95A9F7809539
:0C61E0009095BC01CD010895F894FFCF0C
:1061EC0005EA010000FF2D16CF16A0166416301616
:1061FC00010101E4032808140A321E5F5A313530BC
:10620C00005F3F3F3F3F005F415438340041540032
:10621C005854005445524D494E414C004E4F4E453A
:10622C00004D4F55534500494E54454C4C49004C7C
:10623C004F474954454348004558504C4F524552DE
:10624C000044454641554C5400397F225E07DF0619
:0E625C00BD0662067B069406000800040002E0
:106800008800EA44E944E244040005000600070069
:10681000080009000A000B000C000D000E000F001C
:1068200010001100120013001400150016001700CC
:10683000180019001A001B001C001D001E001F007C
:10684000200021002200230024002500260027002C
:10685000280029002A002B002C002D002E002F00DC
:10686000300031003200330034003500360037008C
:10687000380039003A003B003C003D003E003F003C
:1068800040004100420043004400450046004700EC
:10689000480049004A004B004C004D004E004F009C
:1068A000500051005200530054005500560057004C
:1068B000580059005A005B005C005D005E005F00FC
:1068C0006000610062006300640065A185006700EC
:1068D000680069006A006B006C006D006E006F005C
:1068E0007000710072007300890087008A008B00BD
:1068F000E000E100E200E300E400E500E600E7007C
:106900000100010001000100EA4401000100E2442D
:106910000100010001000100460001004A004B0097
:10692000010001004700480001000100E9440100A6
:106930000100010001000100010001003A003B00DC
:106940003C003D003E003F0040004100420043004B
:10695000010035004C0039000100440045005200A0
:1069600049000100010050004F0029004D004E0079
:1069700051000100010001000100010001000100BF
:1069800001000100010001000100010001000100FF
:1069900001000100010001000100010001004D00A3
:1069A0004A004E004B0001000100010001000100FF
:1069B00001000100010001000100010001000100CF
:1069C00001000100010001000100010001000100BF
:1069D00001000100010001000100010001000100AF
:1069E0000100010001000100490001000100010057
:1069F000010001000100010001000100010001008F
:00000001FF
